:100000003B29FF3FFF3FFF3F03138312A001011C69
:100010000728191F0D28A0010E28A00A20081B3C44
:10002000031C1E2801181228191F1828A0011928BE
:10003000A00A20081B3C031C1E280728A001011C45
:100040001F28191B2528A0012628A00A20081B3CD0
:10005000031C362801182A28191B3028A001312832
:10006000A00A20081B3C031C36281F28080040302B
:10007000031383122102031C53282108443C031C50
:10008000532860302202031C53282208643C031CBE
:10009000532860302302031C53282308643C031CAC
:1000A00053280530A40760302102031C7F28210853
:1000B000643C031C7F2840302202031C6D28220868
:1000C000443C031C6D2860302302031C6D28230868
:1000D000643C031C6D280530A40760302202031C19
:1000E0007F282208643C031C7F2840302302031C25
:1000F0007F282308443C031C7F280530A4073530A3
:100100002102031CAB282108393C031CAB283530E5
:100110002202031C99282208393C031C99285030DC
:100120002302031C99282308543C031C99280330FC
:10013000AB0750302202031CAB282208543C031C9E
:10014000AB2835302302031CAB282308393C031CA1
:10015000AB280430AB0750302102031CC52821080E
:10016000543C031CC52835302202031CC528220834
:10017000393C031CC52835302302031CC52823083D
:10018000393C031CC5280430AB0708000313831255
:10019000B0010330300203183A293608B700370897
:1001A00003191A29B801FA3038020318F92805157D
:1001B0000230DB00FF30DA00DB0BDF28E228DA0B4D
:1001C000DF28DC284A30DA00DA0BE42800000511C9
:1001D0000230DB00FF30DA00DB0BEF28F228DA0B0D
:1001E000EF28EC284A30DA00DA0BF4280000B80ACD
:1001F000D3280430DC00FF30DB00FF30DA00DC0BFA
:1002000002290929DB0B05290829DA0B052902290E
:10021000FF281030DB00FF30DA00DB0B1029132938
:10022000DA0B10290D292630DA00DA0B1529000027
:10023000B703CF281A30DC00FF30DB00FF30DA00D4
:10024000DC0B23292A29DB0B26292929DA0B26296D
:10025000232920297F30DB00FF30DA00DB0B312936
:100260003429DA0B31292E295930DA00DA0B3629F4
:10027000B00AC9280800031383169F0104308312B3
:100280009900A030831699000A30850083128501F9
:100290008316950183308100B10103138316B001E9
:1002A0000C30300203185C293008243FD00050087D
:1002B00084008001B00A5029B001031383163F3037
:1002C000300203187C2904200108B20033083202EE
:1002D000D1005108A1005108A100A10CA1133208BE
:1002E000B30003303002031C762937202308A20014
:1002F0002108A300B00A5D2903138312B401B001E1
:100300000C303002031896293008243F840000087E
:10031000D10051083402031894293008243F840086
:100320000008B4003008B500B00A802934083C3C0D
:100330000318B5293508003A031DA829051431080A
:10034000003A031DA6290230B600C6200130B100D4
:100350003508073A031DB52905103108013A031D78
:10036000B4290130B600C620B1014D29B629FF3F9E
:02400E00C23FAF
:00000001FF
